:04000000B201C2295E
:10000800040864000C1E052899000314BD29B216C3
:10001800B21EB212B2191428B2154D2003183B288B
:100028000830A3006120A20DA30B1628B21E46209B
:100038006B206720B21A3B20402022080310BD29FC
:10004800B216B21EB21232192E28FE39B30032157A
:100058000310BD29321A3628A60032164D2003187F
:100068003B282608542003183B28B21EBD294620E9
:100078006B2032113212B21136088400340884170A
:1000880080044C28360884003409800584178005CC
:10009800080040206B20462067203308B219013839
:1000A800A2000830A300A20D03184020031C46201C
:1000B8006B206720A30B572840206B20360884004C
:1000C80034080005FF3E37088400350949283708F9
:1000D800840035084328A40029080319BD292518D8
:1000E80083172408840000088313B821A40AA903ED
:1000F8007028B31329080319B3170430A800250E74
:100108008A2025088A20240E8A2024080F39F63EE2
:100118000318073E0A3EAD28B31329080319B3177D
:100128000530A8002730A3001030A6200330A30014
:10013800E830A620A3016430A620A3010A30A62037
:100148002408AD28A2002508A1002408A0008621C3
:100158002008A000A8030319B31329080319B72816
:100168002802031808002008031DB313B31B080056
:10017800303EB8290830A600A700370884003508A3
:1001880033190B21331D0D21360884003408102142
:10019800A001A10126080319BD29B31802213608B8
:1001A800840000083405FF3EA00DA10DB31C0221F8
:1001B800A60BD1282708331839292008BD2908306B
:1001C800A60037088400350833190B21331D0D218B
:1001D800360884003409142126080319BD29331868
:1001E800392136088400A10CA00C00083404031C33
:1001F800340680000221A60BF528BD2937088400A3
:1002080035088006000008290929800608008004AE
:100218001329FF3A8005142984178004BD29FF3A61
:1002280084178005BD29A301A200FF30A207031C83
:10023800A307031CBD290330A100E4302521192997
:10024800A101F63EA000A109031C3029FE300000E0
:10025800A00703182B29A0076400A10F2A29000072
:1002680020183629201838290800A201A30140299E
:10027800A10CA00CA20DA30DFF3E03183C292308D6
:10028800A1002208A000BD29A20002305D29A20019
:1002980003305D29A101A301A20001305D29A2005C
:1002A80006305D29A101A301A20004305D29A20046
:1002B8000530A80023082102031D64292208200212
:1002C800043003180130031902302805031DFF30DC
:1002D800BD290038031DFF300405031DFF30BD296B
:1002E8000404031DFF30BD29A2002008A60024082D
:1002F800A0002608A4002108A6002508A1002608B9
:10030800A5008829A501A4011030A600210DA40D7F
:10031800A50D2208A4022308031C230FA502031815
:100328009C292208A40723080318230FA5070310F4
:10033800A00DA10DA60B8A292008BD291030A80000
:10034800A101A001A70CA60C031CB0292208A00734
:1003580023080318230FA107A10CA00CA50CA40CBB
:10036800A80BA6292408BD29840031088A00300872
:100378008200831303138312640008008316073076
:100388009900203098008312903098008316073027
:100398009F00B201B301B001B1018312E201E30190
:1003A800E001E101EA01EB01E801E9018316E50159
:1003B800E90186130613861290308700E60183123E
:1003C800D401D5018316EB01B601B7018312CE0122
:1003D800CF01FC01FD01C401C5010130A300F430C7
:1003E8008A011821861383168613831286128316B0
:1003F80086128312061383160613533083128A015A
:10040800052044308A0105204D308A0105204D30F1
:100418008A01052033308A01052046308A010520EB
:1004280020308A01052044308A01052065308A0180
:1004380005206D308A0105206F308A0105202030A3
:100448008A01052056308A01052065308A01052079
:1004580072308A01052020308A01052031308A0156
:1004680005202E308A01052034308A0105200D3000
:100478008A0105200A308A01052053308A010520A7
:1004880074308A01052061308A01052072308A01A2
:10049800052074308A01052069308A0105206E30F4
:1004A8008A01052067308A0105202E308A0105203F
:1004B8002E308A0105202E308A0105202E308A012F
:1004C80005200A308A0105200D308A0105208A118D
:1004D8000A164E2F0130A300F4308A011821831622
:1004E800E001D601D701543083128A010520723009
:1004F8008A01052079308A01052069308A010520A2
:100508006E308A01052067308A0105202E308A0165
:1005180005202E308A0105202E308A0105200A3058
:100528008A0105200D308A01052007158316FF3042
:10053800E4000A30E20083128A110A12C526071164
:1005480032308A01172183164030E1009530E300EC
:10055800831283166108E40007308312B600203046
:10056800B4000730B7000830B5000130B300831677
:1005780064088312A000A1018A01E3208316E40124
:100588000430E20083128A110A12C5268316630812
:10059800E40007308312B6002030B4000730B700FB
:1005A8000830B5000130B300831664088312A00038
:1005B800A1018A01E32083160130DF0083128A112A
:1005C8000A12D623640083166008013C8A110A12B5
:1005D8008312031D162B4E308A0105206F308A01C5
:1005E800052020308A01052072308A0105206530F7
:1005F8008A01052073308A01052070308A010520A0
:100608006F308A0105206E308A01052073308A0117
:10061800052065308A0105200A308A0105200D3041
:100628008A010520071532308A0117210711640055
:1006380083166008013C8A110A12831203196E2A74
:1006480043308A0105206D308A01052064308A0113
:10065800052030308A01052020308A0105204F30DE
:100668008A0105204B308A0105200A308A010520BD
:100678000D308A0105208316D601D7018312640044
:1006880083166C08003C8A110A1283120319A32BE3
:1006980007158316FF30E40007308312B6002030B8
:1006A800B4000730B7000830B5000130B300831636
:1006B80064088312A000A1018A01E3208A110A12AA
:1006C8008B27071183164130E40007308312B600E8
:1006D8002030B4000730B7000830B5000130B3004F
:1006E800831664088312A000A1018A01E3208316FF
:1006F800E4010430E20083128A110A12C526831627
:10070800FF30E40083128A110A1260278A110A1244
:100718008B278316D60A0319D70A56088312A00016
:10072800831657088312A1000F30A300FF308A01F7
:1007380050218A110A12031D6E2A8A01432B83163F
:10074800FF30E40083124D308A0105204D308A01C4
:10075800052043308A01052020308A0105204930D0
:100768008A0105204E308A01052049308A0105207A
:1007780054308A01052020308A0105204F308A0133
:1007880005204B308A01052021308A0105200A30D6
:100798008A0105200D308A010520861683168612E7
:1007A800831208008316D601D701E0018312640082
:1007B80083166C085F028A110A1283120319062C29
:1007C8000730B6001030B4000730B7000830B50065
:1007D800B3018A01BE208316EC00D60A0319D70A92
:1007E80056088312A000831657088312A100103000
:1007F800A30000308A0150218A110A12031D092C16
:100808008A01DB2B8A110A120D2C83160130E000B5
:10081800831208008617831686138312071583161A
:10082800FF30DE0083128A110A1279278A110A1210
:100838008B27071183165830DA008312470883166E
:10084800DB00831246088316DC00831249088316EE
:10085800DD00831248088316DE0083128A110A120B
:10086800EB268316FF30DE0083128A110A127927DD
:100878008A110A128B278316DF0183128A01D62375
:100888008316FE30DE0083128A110A127927560871
:10089800C4005708C5004408A0004508A10059082D
:1008A800A30058088A0150218A110A12031D8A2CB4
:1008B8000730B6000230B4000730B7000130B50089
:1008C800A0308A01262045088A01262044088A018A
:1008D80026208A010B208316E40007308312B60015
:1008E8002030B4000730B7000830B5000130B3003D
:1008F800831664088312A000A1018A01E320C40AB8
:100908000319C50A8A110A12031D4F2C8316FF30DA
:10091800E4000230E20083128A110A12C5268A1105
:100928000A128B270F3083166C05EF0083128A1189
:100938000A128B27640083166C08003C8A110A127D
:100948008312031DB72C0730B6001030B4000730EF
:10095800B7000830B500B3018A01BE208316EC0049
:1009680083128A019E2C8A110A127F268613831607
:1009780086138312080007158316FF30DE008312E2
:100988008A110A1279278A110A128B2707118316EE
:100998005130DA00831247088316DB0083124608B9
:1009A8008316DC00831249088316DD008312480889
:1009B8008316DE0083128A110A12EB268316FF3093
:1009C800DE0083128A110A1279278A110A128B27EC
:1009D8008316DF0183128A01D62364008316600818
:1009E800013C8A110A128312031D3F2D52308A01DD
:1009F800052065308A01052061308A0105206430B0
:100A08008A01052020308A01052045308A01052009
:100A180072308A01052072308A0105206F308A0100
:100A2800052072308A01052020308A0105205230C5
:100A38008A01052065308A01052073308A01052066
:100A480070308A01052020308A0105206E308A0125
:100A580005206F308A01052074308A010520203076
:100A68008A01052030308A0105200A308A010520D4
:100A78000D308A0105208316FE30DF0083128A01BB
:100A8800D623640083166008013C8A110A12831277
:100A9800031D992D52308A01052065308A010520F1
:100AA80061308A01052064308A01052020308A01DE
:100AB800052045308A01052072308A0105207230F0
:100AC8008A0105206F308A01052072308A010520CD
:100AD80020308A01052052308A01052065308A01BC
:100AE800052073308A01052070308A0105202030E6
:100AF8008A0105206E308A0105206F308A010520A1
:100B080074308A01052020308A01052024308A01AA
:100B1800052046308A01052045308A0105200A3023
:100B28008A0105200D308A0105205608D200570891
:100B3800D3005208A0005308A1005908A300580880
:100B48008A0150218A110A12031DD52D0730B600DB
:100B58001030B4000730B7000830B500B3018A017F
:100B6800BE208316E40007308312B6000230B400BA
:100B78000730B7000130B500A0308A01262053089D
:100B88008A01262052088A012620831664088312C7
:100B98008A012420D20A0319D30A8A110A12031DD2
:100BA8009D2D8A110A128B278A110A128B278A1106
:100BB8000A127F26080083165030E10083128A113A
:100BC8000A12FF25080083166030E10083128A119B
:100BD8000A12FF25080083166130E10083128A118A
:100BE8000A12FF25080083166630E10083128A1175
:100BF8000A12FF25080007158316FF30DE0083124E
:100C08008A110A1279278A110A128B27071183166B
:100C18006108DA00831247088316DB00831246084E
:100C28008316DC00831249088316DD008312480806
:100C38008316DE0083128A110A12EB268316FF3010
:100C4800E4000230E20083128A110A12C5268A11D2
:100C58000A128B278316DF0183128A01D6236400C8
:100C680083166008013C8A110A128312031D7E2E26
:100C780043308A0105206D308A01052064308A01DD
:100C8800052020308A01052065308A010520723050
:100C98008A01052072308A0105206F308A010520FB
:100CA80072308A01052020308A01052052308A01DD
:100CB800052065308A01052073308A0105207030CF
:100CC8008A01052020308A0105206E308A0105201E
:100CD8006F308A01052074308A01052020308A018E
:100CE800052030308A0105200A308A0105200D30A0
:100CF8008A010520080007158316FF30E400073035
:100D08008312B6002030B4000730B7000830B500B1
:100D18000130B300831664088312A000A1018A0180
:100D2800E3208A110A128B27071183164D30DE0043
:100D380083128A110A1279278316E4010430E2002B
:100D480083128A110A12C5268316FF30DE00831229
:100D58008A110A1279270730B6001030B40007301C
:100D6800B7000830B500B30110308A01BF208316E0
:100D7800AE00831221088316AF002E08EB00831201
:100D8800080083160130EF008312640083166F0891
:100D980062028A110A128312031CEA2E0730B60077
:100DA8002030B4000730B7000830B5000130B30078
:100DB800831664088312A000A1018A01E320831628
:100DC800EF0A8A110A128312031DC92E0800073080
:100DD800B6002030B4000730B7000830B500013045
:100DE800B30083165A088312A000A1018A01E320E8
:100DF80083165B088312A000A1018A01E3208316F1
:100E08005C088312A000A1018A01E32083165D0813
:100E18008312A000A1018A01E32083165E088312D1
:100E2800A000A1018A01E32008000730B6002030A5
:100E3800B4000730B7000830B5000130B30083169E
:100E48005B088312A000A1018A01E32083165C08D5
:100E58008312A000A1018A01E32083165D08831292
:100E6800A000A1018A01E32083165E088312A00076
:100E7800A1018A01E32008000730B6002030B40041
:100E88000730B7000830B5000130B30083165C089E
:100E98008312A000A1018A01E32083165D08831252
:100EA800A000A1018A01E32083165E088312A00036
:100EB800A1018A01E32008000730B6002030B40001
:100EC8000730B7000830B5000130B30083165D085D
:100ED8008312A000A1018A01E32083165E08831211
:100EE800A000A1018A01E32008000730B6002030E5
:100EF800B4000730B7000830B5000130B3008316DE
:100F08005E088312A000A1018A01E32008000730CF
:100F1800B6001030B4000730B7000830B500B30190
:100F28008A01BE208316EC0083120800D60108301F
:100F3800D700FF30D8000930D900C601C701C80161
:100F4800C9018A01BF240B30C4000830C50007302E
:100F5800B6000230B4000730B7000130B500A03049
:100F68008A01262045088A01262044088A0126206D
:100F78008A010B20CC000C30C4000830C5000730B3
:100F8800B6000230B4000730B7000130B500A03019
:100F98008A01262045088A01262044088A0126203D
:100FA8008A010B20CD000D30C4000830C500073081
:100FB800B6000230B4000730B7000130B500A030E9
:100FC8008A01262045088A01262044088A0126200D
:100FD8008A010B208316ED0083120E30C4000830FE
:100FE800C5000730B6000230B4000730B700013042
:100FF800B500A0308A01262045088A012620440829
:101008008A0126208A010B208316B40083120F3030
:10101800C4000830C5000730B6000230B4000730FD
:10102800B7000130B500A0308A01262045088A01A2
:10103800262044088A0126208A010B208316B50041
:1010480083121130C4000830C5000730B6000230E2
:10105800B4000730B7000130B500A0308A0126205F
:1010680045088A01262044088A0126208A010B2087
:101078008316AC0083121230C4000830C500073054
:10108800B6000230B4000730B7000130B500A03018
:101098008A01262045088A01262044088A0126203C
:1010A8008A010B208316AD0083121630C400083065
:1010B800C5000730B6000230B4000730B700013071
:1010C800B500A0308A01262045088A012620440858
:1010D8008A0126208A010B20FE001730C400083040
:1010E800C5000730B6000230B4000730B700013041
:1010F800B500A0308A01262045088A012620440828
:101108008A0126208A010B20FF001330C400083012
:10111800C5000730B6000230B4000730B700013010
:10112800B500A0308A01262045088A0126204408F7
:101138008A0126208A010B208316C40083121430EA
:10114800C4000830C5000730B6000230B4000730CC
:10115800B7000130B500A0308A01262045088A0171
:10116800262044088A0126208A010B208316C50000
:10117800C201C30144088312A000831645088312E4
:10118800A100A30100308A015B218A150A12031D00
:1011980035292030C4000830C5000730B6000230B9
:1011A800B4000730B7000130B500A0308A0126200E
:1011B80045088A01262044088A0126208A010B2036
:1011C8008316C40083122130C4000830C5000730DC
:1011D800B6000230B4000730B7000130B500A030C7
:1011E8008A01262045088A01262044088A012620EB
:1011F8008A010B208316C50083122230C4000830F0
:10120800C5000730B6000230B4000730B70001301F
:10121800B500A0308A01262045088A012620440806
:101228008A0126208A010B208316C20083122330EC
:10123800C4000830C5000730B6000230B4000730DB
:10124800B7000130B500A0308A01262045088A0180
:10125800262044088A0126208A010B208316C30011
:10126800831283162C088312A60083162D08831276
:10127800A7002030A200A3018A01A2218316BA0088
:10128800831225088316BB0083124C088316BA07FD
:1012980083124D080318013E8316BB070130BA02BA
:1012A8000030031C013EBB023A088312A0008316DB
:1012B8003B088312A1004C08A2004D08A3008A0134
:1012C80086218316AA00831221088316AB00831295
:1012D8000230A600A7017E08A2007F08A3008A01A9
:1012E800A2218316BA00831225088316BB0034088E
:1012F800BA0735080318013EBB073A082A07A000B9
:101308003B080318013E2B07A10020088312A60002
:10131800831621088312A7004C08A2004D08A300D9
:101328008A01A2218316A400831225088316A5002A
:1013380020088312A600831621088312A7004C08F0
:10134800A2004D08A3008A01A22120088316A2004A
:10135800831221088316A30022088312DC00831657
:1013680023088312DD00831624088312DE00831607
:1013780025088312DF00E001E1014C08A6004D08B2
:10138800A700831634088312A20083163508831237
:10139800A3008A01A221E2002508E3007E08A60036
:1013A8007F08A700A2010230A3008A01A221EA0057
:1013B8002508EB007E08A6007F08A700A2010230DE
:1013C800A3008A01A2212008E8002108E900620898
:1013D800EA0763080318013EEB0764008A150A123E
:1013E800031CF929E80A0319E90A7E08A6007F0800
:1013F800A700A2010230A3008A01A22120088316B7
:10140800B000831221088316B10083127E08A6005B
:101418007F08A700A2010230A3008A01A221831637
:10142800B200831225088316B30083126808831656
:10143800B007831269080318013E8316B1078312A7
:101448006A088316B20783126B080318013E8316D5
:10145800B30764008A150A128312031C382A8316FC
:10146800B00A0319B10A8312831642088312A00036
:10147800831643088312A100A30100308A01532177
:101488008A150A12031D4B2A8A150A127B2A83160B
:1014980020084402BE002108031C013E4502BF008B
:1014A8003E088312A00083163F088312A10083160A
:1014B8006D088312A200A3018A0186218316BE004B
:1014C800831221088316BF003E088312A0008316EA
:1014D8003F088312A1000F30A300F5308A014B2189
:1014E8008A150A12031D7B2A8A150A1615288316DF
:1014F8001030E800831283166D088312A600A70136
:101508004C08A2004D08A3008A01A221D00025089A
:10151800D1000800D6010230D700FF30D8000330D0
:10152800D900831630088312C60083163108831247
:10153800C700831632088312C80083163308831243
:10154800C9008A01BF2483162030C8000230C900B0
:10155800EA01831264000B3083166A028A150A12A4
:1015680083120318DE2A0730B6000230B4000730B1
:10157800B7000130B500A0308A012620831649083B
:1015880083128A0126208316480883128A0126209E
:101598008A010B208316BA006A08383E84003A088C
:1015A8008000C80A0319C90AEA0A8A150A128312AE
:1015B800031DAE2A3808A00040308A014E21831648
:1015C800BA0083123808A0007B308A01562183169E
:1015D800BC003A088312840083163C0883128A01EF
:1015E8006D218A150A12031DA12C0A308A010520D3
:1015F8000D308A0105204E308A0105206F308A019E
:10160800052020308A01052046308A0105206930EE
:101618008A0105206C308A01052065308A01052081
:1016280020308A01052066308A0105206F308A0142
:10163800052075308A0105206E308A010520643046
:101648008A0105202E308A0105202E308A010520C6
:101658002E308A01052063308A01052072308A0104
:10166800052065308A01052061308A010520743023
:101678008A01052069308A0105206E308A0105201B
:1016880067308A01052020308A01052061308A01EF
:10169800052020308A01052066308A01052069303E
:1016A8008A0105206C308A01052065308A010520F1
:1016B80020308A01052044308A01052041308A0102
:1016C800052054308A01052041308A010520303038
:1016D8008A01052030308A01052030308A01052032
:1016E80031308A0105202E308A01052054308A01C4
:1016F800052058308A01052054308A0105200A3017
:101708008A0105200D308A0105208316C8010230A0
:10171800C9008312831648088312A000831649085B
:101728008312A1000330A300FF308A0150218A15DB
:101738000A12031DC02B0730B6000230B400073070
:10174800B7000130B500A0308A0126208316490869
:1017580083128A0126208316480883128A012620CC
:1017680000308A0124208316C80A0319C90A8A1579
:101778000A128312031D8E2B8316C8010230C9007A
:10178800D801D9018312831658088312A000831642
:1017980059088312A100A3013F308A0150218A15FC
:1017A8000A12031D672C831659088A150A12831218
:1017B800031D412C831658083F3C8A150A128312D0
:1017C800031C412C8A150A12EF238316E4008312A6
:1017D8008A150A12412C0C308A0083165808831285
:0217E800002CD3
:101800008207E53441345434413430343034303498
:101810003134543458345434203418349A347B34AA
:1018200061348634313486343134003400347C34CD
:1018300061348634313400340034003400340034F0
:10184000003444344134543441343034303430344E
:101850003134543458345434203418349A347B346A
:101860006134863431348C34313400340034023401
:10187000AB348C343134023400340034003400345E
:1018800000340730B6000230B4000730B700013032
:10189000B500A0308A0126208316490883128A01E8
:1018A00026208316480883128A012620831664089E
:1018B00083128A0124208316C80A0319C90AD80A88
:1018C0000319D90A8A150A128312031DC72B8A111C
:1018D0000A16392183162030C8000230C900EA01F7
:1018E000831264000B3083166A028A150A1283126F
:1018F0000318A12C0730B6000230B4000730B7003F
:101900000130B500A0308A012620831649088312D1
:101910008A0126208316480883128A0126208A011C
:101920000B208316BA006A08383E84003A0880000B
:10193000C80A0319C90AEA0A8A150A128312031D82
:10194000712C0A308A0105200D308A0105204630AD
:101950008A01052069308A0105206C308A01052042
:1019600065308A01052020308A0105204E308A0129
:10197000052061308A0105206D308A01052065301F
:101980008A0105203A308A0105200B30A900043075
:10199000B000B101A50138308A016F200A308A01F8
:1019A00005200D308A0105200730B6000230B40052
:1019B0000730B7000130B500A0308A012620023080
:1019C0008A0126203F308A0126208A010B208316B7
:1019D000A70007308312B6000230B4000730B7000A
:1019E0000130B500A0308A01262002308A0126206D
:1019F0003E308A0126208A010B208316A60007307C
:101A00008312B6000230B4000730B7000130B500D1
:101A1000A0308A01262002308A0126203D308A012A
:101A200026208A010B208316A90007308312B600F6
:101A30000230B4000730B7000130B500A0308A0191
:101A4000262002308A0126203C308A0126208A0185
:101A50000B208316A80007308312B6000230B400B2
:101A60000730B7000130B500A0308A0126200230CF
:101A70008A0126203B308A0126208A010B2083160A
:101A8000B90007308312B6000230B4000730B70047
:101A90000130B500A0308A01262002308A012620BC
:101AA0003A308A0126208A010B208316B8002608C6
:101AB000CC002708CD002808CE002908CF008312CB
:101AC00050088316CA00831251088316CB00831274
:101AD0008A110A16BD230230831652078312DA00D8
:101AE000831653080318013E8312DB00831638085F
:101AF0008312A000831639088312A100A3010030CD
:101B00008A015B218A150A12031DB92D8316023042
:101B1000B800B90107308312B6000230B4000730B4
:101B2000B7000130B500A0308A01262002308A01BA
:101B300026203B308A0126208316390883128A0129
:101B400024200730B6000230B4000730B70001305F
:101B5000B500A0308A01262002308A0126203A30C2
:101B60008A0126208316380883128A012420CE0198
:101B7000CF01831626088312DC0083162708831200
:101B8000DD00831628088312DE00831629088312DD
:101B9000DF00831624088312DE0783162508031846
:101BA000013E8312DF0764008A150A12031CDB2D35
:101BB000DC0A0319DD0A831628088312A0008316A5
:101BC00029088312A100A30100308A015021831645
:101BD000BA0026088312A000831627088312A100EA
:101BE000A30100308A0150218316BC003A088312F9
:101BF000840083163C0883128A0174218316BC007A
:101C0000BD0064003C083D048A150A1283120319C2
:101C1000262E83162608CC002708CD002808CE00E3
:101C20002908CF00831250088316CA008312510876
:101C30008316CB0083128A110A16BD23831650081F
:101C40008312CE00831651088312CF008A150A1220
:101C5000A7268316340883127C028316BA0035083F
:101C6000031C013E83127D028316BB003A088312D7
:101C7000A00083163B088312A1000330A200A30139
:101C80008A01862124088316EE006E0883127C02E6
:101C90008316BA0083127D08031CFF3E8316BB0027
:101CA0003A088312A60083163B088312A7004C084B
:101CB000A2004D08A3008A01A221E6002508E70042
:101CC00083166E0883127C028316BA0083127D0885
:101CD000031CFF3E8316BB003A088312A60083163E
:101CE0003B088312A7004C08A2004D08A3008A01FC
:101CF000A2212008E4002108E5007E08A6007F0854
:101D0000A7004C08A2004D08A3008A01A221EE0002
:101D10002508EF007E08A6007F08A7004C08A20057
:101D20004D08A3008A01A2212008EC002108ED0043
:101D30006608EE0767080318013EEF0764008A157E
:101D40000A12031CA62EEC0A0319ED0A080064000F
:101D5000831668080C3C8A150A128312031DE22EB2
:101D600003105B0CF7005A0CF6005A08F6075B08E4
:101D70000318013EF70764008A150A12031CC62ED9
:101D80000130F400F5018A150A12C82EF401F5019C
:101D90005A08A6005B08A7000330A200A3018A012D
:101DA000A2218316BA00831225088316BB000310F4
:101DB0003B0C8312F30083163A0C8312F2008A154F
:101DC0000A12FF2E5A08A6005B08A7000230A200E4
:101DD000A3018A01A221F6002508F7005A08A600EF
:101DE0005B08A7000230A200A3018A01A2212008FB
:101DF000F4002108F5007608F2007708F300720875
:101E0000A0007308A100A2010630A3008A01862168
:101E10002408D4002508D50074088316CC0083124A
:101E200075088316CD00831276088316CE008312C0
:101E300077088316CF0083124C088316CA008312DA
:101E40004D088316CB0083128A110A16BD23831610
:101E5000520834078312FC00831653080318013E0E
:101E600035078312FD007C08A6007D08A7004C08FA
:101E7000A2004D08A3008A01A221E2002508E30088
:101E80007C08A6007D08A7004C08A2004D08A3000E
:101E90008A01A2212008E0002108E1007E08A600B6
:101EA0007F08A7004C08A2004D08A3008A01A221C8
:101EB000EA002508EB007E08A6007F08A7004C0872
:101EC000A2004D08A3008A01A2212008E8002108F1
:101ED000E9006208EA0763080318013EEB076400A3
:101EE0008A150A12031C772FE80A0319E90A080069
:101EF000D6011030D700FF30D8001130D900640867
:101F0000C6006508C7006608C8006708C9008A01DE
:101F1000BF24D6011230D700FF30D8001330D900CB
:101F20000030C80702300318013EC90764008A1553
:101F30000A12031C9E2FC60A0319C70A8A01BF246E
:101F4000D6011430D700FF30D8001530D90000304A
:101F50006607C80004300318013E6707C900640023
:101F60008A150A12031CB72FC60A0319C70A8A0169
:101F7000BF24080083165030E1008312C601C70158
:101F80004A08C8004B08C9008A01FF2508005E08FE
:101F9000A0005F08A100FF30A300FF308A015B2191
:101FA0008A150A12031DDC2FDC0A0319DD0ADE0183
:101FB000DF018A150A12DF2FDE0A0319DF0A080083
:101FC000831628088312A000831629088312A10013
:101FD000FF30A300FF308A015B218A150A12031D1E
:101FE000FB2F8316A60A0319A70AA801A9018312C9
:101FF0008A110A1600288316A80A0319A90A83124F
:1020000008000730B6000230B4000730B7000130D6
:10201000B500A0308A0126208316370883128A0172
:1020200026208316360883128A0126208316650827
:1020300083128A0124208316B60A0319B70A831271
:10204000CE0A0319CF0A8A150A12E0274E08A0000B
:102050004F08A1005108A30050088A015B218A1192
:102060000A16031D7A288A110A16C8225808A000E9
:102070005908A1001530A300FF308A015B218A11A5
:102080000A16031D472883160130E60083128A11C1
:102090000A165321640083166608013C8A110A1649
:1020A0008312031D72280030E60706300318013E34
:1020B000E70764008A110A16031C6128E40A031961
:1020C000E50A0030EE0706300318013EEF07640012
:1020D0008A110A16031C6F28EC0A0319ED0A8A15E7
:1020E0000A127827DA0A0319DB0ACE01CF01831618
:1020F000E6018312831636088312A0008316370880
:102100008312A1000230A30000308A015B218A11F2
:102110000A16031D38290730B6000230B400073014
:10212000B7000130B500A0308A01262002308A01B4
:1021300026203F308A0126208316270883128A0131
:1021400024200730B6000230B4000730B700013059
:10215000B500A0308A01262002308A0126203E30B8
:102160008A0126208316260883128A01242007303C
:10217000B6000230B4000730B7000130B500A0301F
:102180008A01262002308A0126203D308A0126203D
:102190008316290883128A0124200730B6000230F2
:1021A000B4000730B7000130B500A0308A01262006
:1021B00002308A0126203C308A0126208316280816
:1021C00083128A0124205C08831622078312C6002A
:1021D0005D080318013E831623078312C7005E08BB
:1021E000A0005F08A100A2010230A3008A0186219D
:1021F00024088316BA00831225088316BB003A0808
:1022000083125E02C80083163B08031C013E831242
:102210005F02C900D601D701FF30D8000130D900D4
:102220008A010E245E08A0005F08A100FD30A30013
:10223000FF308A0153218A110A16031D2B29DC0A5B
:102240000319DD0A0030DE0702300318013EDF0704
:102250008A110A1631290030DE0702300318013EC8
:10226000DF078316B601B70183128A110A163921D6
:102270000800D6010230D700FF30D8000330D90063
:10228000831630088312C600831631088312C700F4
:10229000831632088312C800831633088312C900DC
:1022A0008A010E2408008A150A12A7260A308A011C
:1022B00005200D308A01052046308A010520613055
:1022C0008A01052074308A01052053308A010520D7
:1022D00065308A01052063308A0105203A308A0181
:1022E00005200430A9007C08A4007D08A500043066
:1022F000B000B1018A017D2020308A0105204630DE
:102300008A01052061308A01052074308A01052088
:1023100031308A0105203A308A0105200430A900B5
:102320006408A4006508A5000430B000B1018A016A
:102330007D200430A9006608A4006708A5000430C9
:10234000B000B1018A017D2020308A0105204F3084
:102350008A01052066308A01052066308A01052041
:1023600053308A01052065308A01052074308A01C6
:1023700005203A308A0105200430A9005408A40041
:102380005508A5000430B000B1018A017D2020303D
:102390008A01052045308A01052041308A01052047
:1023A00064308A01052064308A0105200430A900C8
:1023B0005608A4005708A5000430B000B1018A01F6
:1023C0007D200430A9005808A4005908A500043055
:1023D000B000B1018A017D20D6011030D700FF3056
:1023E000D8001130D9006408C6006508C700660827
:1023F000C8006708C9008A010E246C08C6006D0871
:10240000C7006E08C8006F08C9008A010E2420307A
:102410008A01052046308A01052061308A010520A5
:1024200074308A01052032308A0105203A308A0151
:1024300005200430A9004608A4004708A500043080
:10244000B000B1018A017D200430A9004808A40031
:102450004908A5000430B000B1018A017D200D308B
:102460008A0105200A308A010520D6011230D700E2
:10247000FF30D8001330D9006408C6006508C700D3
:1024800000306607C80002300318013E6707C90024
:1024900064008A110A16031C502AC60A0319C70AC7
:1024A0008A010E246C08C6006D08C70000306E0754
:1024B000C80002300318013E6F07C90064008A118A
:1024C0000A16031C662AC60A0319C70A8A010E24C3
:1024D000D6011430D700FF30D8001530D900640879
:1024E000C6006508C70000306607C800043003183E
:1024F000013E6707C90064008A110A16031C832A7B
:10250000C60A0319C70A8A010E246C08C6006D08A2
:10251000C70000306E07C80004300318013E6F0783
:10252000C90064008A110A16031C992AC60A0319F5
:10253000C70A8A010E240800D2011030D3005208C5
:10254000A0005308A1001530A300FF308A015021DC
:102550008A110A16031DC72A0730B6000230B400DC
:102560000730B7000130B500A0308A01262053089B
:102570008A01262052088A01262000308A01242060
:10258000D20A0319D30A8A110A16031D9F2A0800CA
:102590005A08A6005B08A7000230A200A3018A0126
:1025A000A221F2002508F3007208A0007308A10020
:1025B000A2010630A3008A0186212408D400250840
:1025C000D50000305407D60010300318013E5507DF
:1025D000D70001305607D80057080318013ED9002C
:1025E0005808A0005908A1001530A300FF308A0147
:1025F0005B218A110A16031D372B01305A078316F7
:10260000C00083125B080318013E8316C100073027
:102610008312B6000230B4000730B7000130B500B5
:10262000A0308A01262057088A01262056088A01F0
:1026300026208316400883128A0124200730B60022
:102640000230B4000730B7000130B500A0308A0175
:10265000262059088A01262058088A012620831638
:10266000410883128A0124208A110A16782B073028
:10267000B6000230B4000730B7000130B500A0301A
:102680008A01262057088A01262056088A0126201A
:10269000FF308A0124200730B6000230B400073032
:1026A000B7000130B500A0308A01262059088A0100
:1026B000262058088A012620FF308A0124205A0843
:1026C000A0005B08A100A30102308A0148218A1101
:1026D0000A16031DBC2B5608A0005708A100103095
:1026E000A30000308A0148218A110A16031DBC2B61
:1026F0000730B6000230B4000730B7000130B50033
:10270000A0308A012620023056028316BA0000301B
:10271000031C013E831257028316BB003B08831241
:102720008A01262083163A0883128A0126205A0835
:102730008A0124200730B6000230B4000730B70009
:102740000130B500A0308A012620023058028316DD
:10275000BA000030031C013E831259028316BB00ED
:102760003B0883128A01262083163A0883128A01C5
:1027700026205B088A012420080083164C08831257
:10278000A00083164D088312A10083164E08831201
:10279000A40083164F088312A50083164B088312EA
:1027A000A30083164A0883128A0178218316D20077
:1027B000831221088316D300831224088316D000C5
:1027C000831225088316D100831208000A308A017B
:1027D00005200D308A01052043308A0105206C3028
:1027E0008A01052075308A01052073308A01052091
:1027F0003A308A0105200430A9007008A40071084D
:10280000A5000430B000B1018A017D2020308A018A
:10281000052045308A01052061308A010520643099
:102820008A01052064308A01052072308A01052062
:102830003A308A0105200430A9005608A400570840
:10284000A5000430B000B1018A017D2020308A014A
:1028500005204F308A01052066308A010520663048
:102860008A01052053308A01052065308A01052040
:1028700074308A0105203A308A0105200430A9000D
:102880007208A4007308A5000430B000B1018A01E9
:102890007D200A308A0105200D308A0105200800BC
:1028A000D601D701FF30D8000130D900C601C701D9
:1028B000C801C9018A016E228A019A270D308A0156
:1028C00005200A308A01052042308A010520503057
:1028D0008A01052053308A0105203D308A010520F8
:1028E0000430A9004C08A4004D08A5000430B00035
:1028F000B1018A017D200D308A0105200A308A014C
:10290000052053308A01052050308A0105204330CC
:102910008A0105203D308A0105200430A900831674
:102920006D088312A400A5010430B000B1018A0132
:102930007D200D308A0105200A308A0105205230A1
:102940008A01052053308A01052043308A01052081
:102950003D308A0105200430A90083163408831213
:10296000A400831635088312A5000430B000B1011D
:102970008A017D200D308A0105200A308A01052058
:1029800052308A01052045308A01052043308A01F2
:1029900005203D308A0105200430A90083162C084B
:1029A0008312A40083162D088312A5000430B00002
:1029B000B1018A017D200D308A0105200A308A018B
:1029C000052046308A01052041308A010520543017
:1029D0008A01052020308A01052073308A010520F4
:1029E00065308A01052063308A01052073308A0131
:1029F00005203D308A0105200430A9007E08A4008E
:102A00007F08A5000430B000B1018A017D200D309F
:102A10008A0105200A308A01052054308A010520E8
:102A20004F308A01052053308A0105203D308A014C
:102A300005200430A900831642088312A4008316DF
:102A400043088312A5000430B000B1018A017D2043
:102A50000430A900831644088312A4008316450895
:102A60008312A5000430B000B1018A017D200D3031
:102A70008A0105200A308A01052052308A0105208A
:102A800044308A01052053308A0105203D308A01F7
:102A900005200430A90083162A088312A400831697
:102AA0002B088312A5000430B000B1018A017D20FB
:102AB0000D308A0105200A308A01052046308A013E
:102AC000052044308A01052053308A0105203D301D
:102AD0008A0105200430A900831620088312A4006F
:102AE000831621088312A5000430B000B1018A01C9
:102AF0007D200D308A0105200A308A0105204630EC
:102B00008A0105205F308A0105204F308A010520A7
:102B100072308A01052069308A01052067308A01F8
:102B200005203D308A0105200430A9005C08A4007E
:102B30005D08A5000430B000B1018A017D20043099
:102B4000A9005E08A4005F08A5000430B000B10130
:102B50008A017D200D308A0105200A308A01052076
:102B600046308A01052041308A01052054308A010F
:102B7000052031308A0105205F308A01052061304F
:102B80008A01052064308A01052064308A0105200D
:102B900072308A0105203D308A0105200430A900E9
:102BA0006008A4006108A5000430B000B1018A01EA
:102BB0007D200430A9006208A4006308A500043049
:102BC000B000B1018A017D200D308A0105200A3054
:102BD0008A01052046308A01052041308A010520FE
:102BE00054308A01052032308A0105205F308A0185
:102BF000052061308A01052064308A010520643097
:102C00008A01052072308A0105203D308A010520A5
:102C10000430A9006808A4006908A5000430B000C9
:102C2000B1018A017D200430A9006A08A4006B0864
:102C3000A5000430B000B1018A017D200D308A0169
:102C400005200A308A01052052308A0105206F30A4
:102C50008A0105206F308A01052074308A01052021
:102C600044308A01052069308A01052072308A01CA
:102C700005205F308A01052061308A01052064301B
:102C80008A01052064308A01052072308A010520FE
:102C90003D308A0105200430A900831630088312D4
:102CA000A400831631088312A5000430B000B101DE
:102CB0008A017D200430A900831632088312A40003
:102CC000831633088312A5000430B000B1018A01D5
:102CD0007D200D308A0105200A308A01052043300D
:102CE0008A0105206C308A01052075308A01052093
:102CF00073308A01052074308A01052065308A010D
:102D0000052072308A0105205F308A01052073306A
:102D10008A01052069308A0105207A308A01052060
:102D200065308A0105203D308A0105200430A90064
:102D30005008A4005108A5000430B000B1018A0178
:102D40007D200D308A0105200A308A0105204C08BB
:102D5000A0004D08A100A30100308A015B218A1167
:102D60000A16031DF82E0A308A0105200D308A014B
:102D7000052045308A01052072308A010520723015
:102D80008A0105206F308A01052072308A010520F2
:102D900020308A01052052308A01052065308A01E1
:102DA000052061308A01052064308A0105206930E0
:102DB0008A0105206E308A01052067308A010520CE
:102DC00020308A01052043308A01052061308A01C4
:102DD000052072308A01052064308A0105200D30FB
:102DE0008A0105200A308A0105208A150A1615284D
:102DF00042308A0105204F308A0105204F308A0178
:102E0000052054308A01052020308A0105204F30EA
:102E10008A0105204B308A0105200A308A010520ED
:102E20000D308A0105208A150A128E2244308A014B
:102E3000052049308A01052052308A0105202030C2
:102E40008A0105204F308A0105204B308A01052078
:102E50000A308A0105200D308A0105208A150A12E0
:102E6000782746308A01052041308A0105205430F8
:102E70008A01052020308A0105204F308A01052073
:102E80004B308A0105200A308A0105200D308A0165
:102E900005208316B601B701831208008A110A16AD
:102EA000502446308A01052041308A0105205430E3
:102EB0008A0105200230A900831668088312A40045
:102EC000A5010430B000B1018A0190200A308A01C6
:102ED00005200D308A01052057308A010520723007
:102EE0008A01052069308A01052074308A01052095
:102EF00069308A0105206E308A01052067308A0119
:102F0000052020308A01052074308A0105206530B3
:102F10008A01052073308A01052074308A0105205A
:102F200020308A01052041308A01052053308A0172
:102F3000052043308A01052049308A0105204930A7
:102F40008A01052020308A01052064308A0105208D
:102F500061308A01052074308A01052061308A01C0
:102F600005202E308A0105202E308A0105202E30C2
:102F70008A0105200A308A0105200D308A010520CA
:102F800083162130E5000130D400D5018312831669
:102F900054088312A000831655088312A100A301D0
:102FA00020308A0150218A150A16031D1228831623
:102FB000D801D9018312831658088312A000831602
:102FC00059088312A1000130A300FF308A0150216B
:102FD0008A150A16031D06288A110A16012083166F
:102FE000E50A64007F3065028A110A168312031C09
:102FF000FD2F83162130E50083128316D80A0319AA
:10300000D90A8A110A168312031DDB2F2E308A017A
:1030100005208316D40A0319D50A8A110A168312C9
:10302000031DC72F8A150A167B280A308A0105203E
:103030000D308A01052055308A0105206E308A0145
:10304000052061308A01052062308A0105206C303C
:103050008A01052065308A01052020308A0105207B
:1030600074308A0105206F308A01052020308A01E2
:10307000052072308A01052065308A010520613003
:103080008A01052064308A01052020308A0105204C
:1030900063308A01052061308A01052072308A017F
:1030A000052064308A0105202E308A0105202E304B
:1030B0008A0105202E308A01052041308A01052031
:1030C00062308A0105206F308A01052072308A0142
:1030D000052074308A01052065308A01052064309E
:1030E0008A01052021308A0105200D308A01052042
:1030F0000A308A0105200A308A0105200D308A0134
:10310000052044308A0105204F308A0105204E30C9
:103110008A01052045308A01052021308A010520D9
:1031200064008A150A16902863008A150A169428E6
:02400E003D3D36
:00000001FF
